:100000000C94AA000C94B4000C94B4000C94B400AA
:100010000C94B4000C94B4000C94B4000C94B40090
:100020000C94B4000C94B4000C94B4000C94B40080
:100030000C94B4000C94B4000C94B4000C94B40070
:100040000C94B4000C94B4000C94B4000C94B40060
:100050000C94B4007F8285888B8F9295989B9EA18B
:10006000A4A7AAADB0B2B5B8BBBDC0C3C5C8CBCDFF
:10007000CFD2D4D6D9DBDDDFE1E3E5E7E8EAECED8A
:10008000EFF0F2F3F4F5F6F8F8F9FAFBFBFCFDFDFE
:10009000FDFEFEFEFEFEFEFEFDFDFDFCFCFBFAFA93
:1000A000F9F8F7F6F5F3F2F1EFEEECEBE9E7E5E35B
:1000B000E1E0DDDBD9D7D5D2D0CECBC9C6C3C1BE36
:1000C000BBB9B6B3B0ADAAA7A4A19E9B9895928FD9
:1000D0008C898683807D797673706D6A6764615ED2
:1000E0005B5855524F4C494744413E3C39373432B6
:1000F0002F2D2A282624221F1D1B1A18161413110F
:100100000F0E0D0B0A09080706050403030202017E
:1001100001000000000000000101010202030404CC
:1001200005060708090A0C0D0E1011131516181AEA
:100130001C1E20222427292B2D303235373A3D3FF3
:100140004245484A4D505356595C5F6265686B6E34
:100150007174777A11241FBECFE5D8E0DEBFCDBF22
:100160000E94BB000C94FD000C94000083B78966CC
:1001700083BFBB9A089583B7896683BFBB9A51E05A
:10018000A3E3B0E05333D0F4252F30E0BD01621B70
:10019000730B40E0E4E5F0E084918CBFC901019766
:1001A000F1F7319681E0E335F807B1F74F5F842F1F
:1001B00090E08617970774F35F5FE4CF61E070E02B
:1001C00040E09D01261B370BE4E5F0E084918CBFF5
:1001D000C9010197F1F7319681E0E335F807B1F7EE
:1001E0004F5F842F90E08617970774F36F5F7F4F00
:0E01F0006233710529F751E0C7CFF894FFCFB5
:00000001FF
